:020000040000FA
:04080000BBEF06F054
:1008100003B218EF05F0F2B433EF05F09EB03BEFF2
:1008200005F09EB243EF05F0F2A81AEF04F0F2B221
:1008300025EF04F0F2A620EF04F0F2B022EF04F06E
:1008400099EF06F0F296F290FF00CD90F2929EA002
:100850002FEF04F00101463F2FEF04F0472B81C139
:1008600085F182C186F183C187F184C188F17DC1A0
:1008700081F17EC182F17FC183F180C184F179C1B0
:100880007DF17AC17EF17BC17FF17CC180F175C1C0
:1008900079F176C17AF177C17BF178C17CF171C1D0
:1008A00075F172C176F173C177F174C178F16DC1E0
:1008B00071F16EC172F16FC173F170C174F169C1F0
:1008C0006DF16AC16EF16BC16FF16CC170F1CECF89
:1008D00069F1CFCF6AF146C16BF147C16CF1CF6AC4
:1008E000CE6A0101466B476B9E90CD800EBC0E8E8A
:1008F0000EBA7EEF04F00E8A99EF06F00E8C0EBE53
:10090000BAEF04F069C16DF16AC16EF16BC16FF1AC
:100910006CC170F16DC171F16EC172F16FC173F193
:1009200070C174F171C175F172C176F173C177F163
:1009300074C178F175C179F176C17AF177C17BF133
:1009400078C17CF179C17DF17AC17EF17BC17FF103
:100950007CC180F17DC181F17EC182F17FC183F1D3
:1009600080C184F181C185F182C186F183C187F1A3
:1009700084C188F10101516B526B536B546B695107
:1009800051276A5152236B5153236C5154236D519B
:1009900051276E5152236F5153237051542371517B
:1009A000512772515223735153237451542375515B
:1009B000512776515223775153237851542379513B
:1009C00051277A5152237B5153237C5154237D511B
:1009D00051277E5152237F515323805154238151FB
:1009E00051278251522383515323845154238551DB
:1009F0005127865152238751532388515423D8902D
:100A00005433533352335133D890543353335233D6
:100A10005133D890543353335233513369C151F168
:100A20006AC152F16BC153F16CC154F199EF06F0F8
:100A30000392030103EE00F080517F0BE92604C00E
:100A4000EFFF802B8151805D700BD8A48B8200005A
:100A50008051815D700BD8A48B9281518019D8B4DC
:100A6000079099EF06F0F2940101383F99EF06F0F4
:100A7000392B99EF06F09E900101463F99EF06F061
:100A8000472B99EF06F09E9204005CA148EF05F019
:100A9000077C07AC63EF05F0C274C2B45DEF05F0EC
:100AA000C3CFADF5C4CFAEF50501D890AE33AD33AD
:100AB000D890AE33AD3364EF05F0C3CF48F1C4CF67
:100AC00049F164EF05F0C28207B491EF05F03AC135
:100AD0003EF13BC13FF13CC140F13DC141F151C14B
:100AE00055F152C156F153C157F154C158F1ADC53A
:100AF000AFF5AEC5B0F5AFC5B1F5B0C5B2F5010102
:100B000048514E2749514F23E86A50230D2E91EF4B
:100B100005F04FC14AF150C14BF14E6B4F6B506B1A
:100B2000078E0201002F99EF06F03C0E006F0501C1
:100B30002951000A7FE005012951010A1BE0050146
:100B40002951020A58E005012951030A54E0050120
:100B50002951040A50E005012951050A4CE005011C
:100B60002951060A48E005012951070A44E0296B8A
:100B70001AEF06F005014D67C5EF05F04E67C5EFAA
:100B800005F04F67C5EF05F05067C9EF05F01AEFA4
:100B900006F051C500F152C501F153C502F154C52B
:100BA00003F10101010E046F000E056F000E066FC8
:100BB000000E076F5CEC1AF000C151F501C152F54F
:100BC00002C153F503C154F50067EEEF05F001676C
:100BD000EEEF05F00267EEEF05F003671AEF06F09F
:100BE0004DC551F54EC552F54FC553F550C554F599
:100BF0000E881AEF06F005012A6701EF06F01AEFDA
:100C000006F00EBE09EF06F00FB009EF06F00EEF8A
:100C100006F007AE0EEF06F017EF06F005012B2FDA
:100C20001AEF06F03C0E2B6F2A2F1AEF06F0050183
:100C30002A6B0E88050105015C6B2DB721EF06F0CC
:100C40005C8101015D672CEF06F05E672CEF06F01A
:100C50005F672CEF06F0606730EF06F060EF06F09C
:100C600061C100F162C101F163C102F164C103F12C
:100C70000101010E046F000E056F000E066F000EDD
:100C8000076F5CEC1AF000C161F101C162F102C1B1
:100C900063F103C164F1006755EF06F0016755EF9A
:100CA00006F0026755EF06F0036760EF06F05DC1DE
:100CB00061F15EC162F15FC163F160C164F10E80F8
:100CC000D57ED5BE34D0D6CF3AF1D7CF3BF138C19F
:100CD0003CF1E86AE8CF3DF10F80010147A77DEFC5
:100CE00006F00E9A0E9C0E9E0101000E516F600ED2
:100CF000526F3D0E536F080E546F01013ABF8DEFD6
:100D000006F03B678DEF06F03C678DEF06F03D6720
:100D10008DEF06F0F28892EF06F0F298516B526B6D
:100D2000536B546BD76AD66A0101386B396B99EFF4
:100D300006F002C0E0FF005001C0D8FF1000A6B2CC
:100D40009FEF06F00CC0A9FF0BC0A8FFA69EA69CB3
:100D5000A684F29E550EA76EAA0EA76EA682F28EEC
:100D6000A694A6B2B1EF06F01200A96EA69EA69CAC
:100D7000A680A8501200076A0E6A0F6A0F010D0EB6
:100D8000C16E860EC06E030EC26E0F01280E896EF4
:100D9000130E926E080E8A6EF30E936E8B6A900E8F
:100DA000946EF18EF19E0D6A01014E6B4F6B506B8C
:100DB0004A6B4B6B0F01280ED56EF28AB00ECD6ECA
:100DC0009D800101516B526B536B546B556B566B8D
:100DD000576B586B596B5A6B5B6B5C6B0E9A0E9C26
:100DE0000E9E760ECA6E9D8202013C0E006FCC6A8A
:100DF000160EB5EC06F0E8CF00F1170EB5EC06F0D4
:100E0000E8CF01F1180EB5EC06F0E8CF02F1190EAB
:100E1000B5EC06F0E8CF03F1010103AF2AEF07F0CC
:100E200053EC1BF0160E0C6E00C10BF09FEC06F09D
:100E3000170E0C6E01C10BF09FEC06F0180E0C6E35
:100E400002C10BF09FEC06F0190E0C6E03C10BF003
:100E50009FEC06F000C15DF101C15EF102C15FF1DE
:100E600003C160F100C161F101C162F102C163F12E
:100E700003C164F11A0EB5EC06F0E8CF00F11B0EC9
:100E8000B5EC06F0E8CF01F11C0EB5EC06F0E8CFAA
:100E900002F11D0EB5EC06F0E8CF03F1010103AF3E
:100EA00080EF07F053EC1BF01A0E0C6E00C10BF034
:100EB0009FEC06F01B0E0C6E01C10BF09FEC06F0D0
:100EC0001C0E0C6E02C10BF09FEC06F01D0E0C6E9A
:100ED00003C10BF09FEC06F01A0EB5EC06F0E8CF5C
:100EE00000F11B0EB5EC06F0E8CF01F11C0EB5ECDD
:100EF00006F0E8CF02F11D0EB5EC06F0E8CF03F1E5
:100F000000C165F101C166F102C167F103C168F179
:100F1000240EAC6E900EAB6E240EAC6E080EB86E46
:100F2000000EB06E1F0EAF6E0401806B816B0F015F
:100F3000900EAB6E0F019D8A0301806B816BA26BDB
:100F40008B9204EC1EF0200EB5EC06F0E8CF29F5EC
:100F500005012951FF0AD8A4B5EF07F0296B200E2F
:100F60000C6E29C50BF09FEC06F00501060E2A6FEA
:100F70002B6B250EB5EC06F0E8CF00F1260EB5EC94
:100F800006F0E8CF01F1270EB5EC06F0E8CF02F14C
:100F9000280EB5EC06F0E8CF03F1010103AFEBEF4B
:100FA00007F053EC1BF0250E0C6E00C10BF09FEC0C
:100FB00006F0260E0C6E01C10BF09FEC06F0270E1A
:100FC0000C6E02C10BF09FEC06F0280E0C6E03C1F4
:100FD0000BF09FEC06F000C14DF501C14EF502C1CA
:100FE0004FF503C150F500C151F501C152F502C1E1
:100FF00053F503C154F5290EB5EC06F0E8CF55F5CD
:1010000005015651555DD8A055C556F50501295124
:10101000020A0EE181B818EF08F00501562F15EF0E
:1010200008F055C556F518EF08F081BA23EF21F006
:10103000210EB5EC06F0E8CF00F1220EB5EC06F07B
:10104000E8CF01F1230EB5EC06F0E8CF02F1240E53
:10105000B5EC06F0E8CF03F1010103AF5EEF08F055
:1010600053EC1BF0210E0C6E00C10BF09FEC06F050
:10107000220E0C6E01C10BF09FEC06F0230E0C6EDD
:1010800002C10BF09FEC06F0240E0C6E03C10BF0B6
:101090009FEC06F0210EB5EC06F0E8CF00F1220E31
:1010A000B5EC06F0E8CF01F1230EB5EC06F0E8CF81
:1010B00002F1240EB5EC06F0E8CF03F100C157F5BC
:1010C00001C158F502C159F503C15AF5AEEC1DF046
:1010D00070EC1CF0C0EC1BF005012951030A12E072
:1010E00005012951040A1DE005012951050A24E0E2
:1010F00005012951060A32E005012951070A38E0A5
:10110000C1EF08F0A6C500F101010F0E00170101A3
:101110000051000A36E001010051050A32E0BEEF3D
:1011200008F0A6C500F101010F0E001701010051E2
:10113000000A27E0BEEF08F00501A651000A21E0F1
:101140000501A651150A1DE00501A651300A19E056
:101150000501A651450A15E0BEEF08F00501A651AC
:10116000000A0FE00501A651300A0BE0BEEF08F0BF
:101170000501A651000A05E0BEEF08F081BA23EF91
:1011800021F007900001F28EF28C07B0F5EF17F016
:101190000EB033EF13F00EB86FEF0DF00301805176
:1011A00081197F0BD8B4F5EF17F013EE00F08151E1
:1011B0007F0BE126812BE7CFE8FFE00BD8B4F5EFFA
:1011C00017F023EE82F0A2511F0BD926E7CFDFFFE5
:1011D000A22BDF50780AD8A4F5EF17F0078061C181
:1011E00000F162C101F163C102F164C103F10101C7
:1011F000040E046F000E056F000E066F000E076FE1
:101200005CEC1AF000AF0EEF09F00101030E616F04
:10121000000E626F000E636F000E646F0301825157
:10122000720AD8B433EF13F08251520AD8B433EFB4
:1012300013F08251630AD8B4B1EF14F08251690AF5
:10124000D8B438EF10F082517A0AD8B44BEF11F0CD
:101250008251490AD8B4D7EF0FF08251500AD8B45E
:10126000F5EF0EF08251700AD8B438EF0FF08251CA
:10127000540AD8B463EF0FF08251740AD8B4A9EFBE
:101280000FF08251730AD8B463EF12F08251530AFF
:10129000D8B4C8EF12F082514C0AD8B465EF09F007
:1012A000E6EF14F0040114EE00F080517F0BE1260C
:1012B00082C4E7FF802B12000D0E826F52EC09F002
:1012C0000A0E826F52EC09F0120003018351300ABA
:1012D000D8B4FCEF0BF003018351310AD8B44AEFC4
:1012E0000CF003018351320AD8B49AEF0CF00301D9
:1012F0008351330AD8B49EEF0CF003018351340AB2
:10130000D8B4ACEF0CF003018351350AD8B474EFB4
:101310000DF0030183514D0AD8B475EF0AF00301B3
:1013200083516D0AD8B48FEF0AF003018351490A43
:10133000D8B474EF0EF003018351500AD8B4A6EF6D
:101340000DF003018351540AD8B41FEF0EF00301CE
:101350008351630AD8B4AFEF0AF003018351430A03
:10136000D8B4A7EF0BF003018351730AD8B4ADEFE3
:101370000AF003018351610AD8B4C2EF09F0D8A47E
:10138000E6EF14F004014C0E826F52EC09F00401F8
:10139000610E826F52EC09F070EC1CF004012C0E0F
:1013A000826F52EC09F053EC1BF0A5C500F101016E
:1013B000F6EC1AF025C182F40401300E822752ECBB
:1013C00009F026C182F40401300E822752EC09F0A4
:1013D00027C182F40401300E822752EC09F0040187
:1013E0002C0E826F52EC09F053EC1BF0A6C500F1F5
:1013F0000101F6EC1AF025C182F40401300E8227B7
:1014000052EC09F026C182F40401300E822752EC1E
:1014100009F027C182F40401300E822752EC09F052
:1014200004012C0E826F52EC09F053EC1BF0A7C59F
:1014300000F10101F6EC1AF025C182F40401300E2E
:10144000822752EC09F026C182F40401300E822773
:1014500052EC09F027C182F40401300E822752ECCD
:1014600009F004012C0E826F52EC09F053EC1BF0D2
:10147000A8C500F10101F6EC1AF025C182F40401BF
:10148000300E822752EC09F026C182F40401300E9E
:10149000822752EC09F027C182F40401300E822722
:1014A00052EC09F004012C0E826F52EC09F053EC5F
:1014B0001BF0ADC500F10101F6EC1AF025C182F474
:1014C0000401300E822752EC09F026C182F4040197
:1014D000300E822752EC09F027C182F40401300E4D
:1014E000822752EC09F0A2EF0DF094EC1BF084C3BC
:1014F00027F1A1EC1BF018EC1BF0200E0C6E00C1C4
:101500000BF09FEC06F000C129F505012951000AF6
:1015100006E005012951010A02E016EC1DF0040164
:101520004C0E826F52EC09F004014D0E826F52ECAA
:1015300009F004012C0E826F52EC09F053EC1BF001
:1015400029C500F1F6EC1AF027C182F40401300E2F
:10155000822752EC09F0A2EF0DF023EF21F00401F5
:101560004C0E826F52EC09F00401630E826F52EC54
:1015700009F0C0EC1BF004012C0E826F52EC09F054
:10158000C4EC0AF0A2EF0DF053EC1BF0ABC500F178
:101590000101003B0F0E0017F6EC1AF027C182F490
:1015A0000401300E822752EC09F0ABC500F10101B5
:1015B0000F0E01010017F6EC1AF027C182F40401A6
:1015C000300E822752EC09F004012D0E826F52EC8E
:1015D00009F0AAC500F10101003B0F0E0017F6EC5F
:1015E0001AF027C182F40401300E822752EC09F070
:1015F000AAC500F101010F0E01010017F6EC1AF067
:1016000027C182F40401300E822752EC09F0040154
:101610002D0E826F52EC09F0A9C500F10101003BCB
:101620000F0E0017F6EC1AF027C182F40401300EF9
:10163000822752EC09F0A9C500F101010F0E01014A
:101640000017F6EC1AF027C182F40401300E82274D
:1016500052EC09F00401200E826F52EC09F0A8C58B
:1016600000F10F0E01010017F6EC1AF027C182F409
:101670000401300E822752EC09F00401200E826F23
:1016800052EC09F0A7C500F101010101003B0F0E6A
:101690000017F6EC1AF027C182F40401300E8227FD
:1016A00052EC09F0A7C500F101010F0E010100176E
:1016B000F6EC1AF027C182F40401300E822752ECB6
:1016C00009F004013A0E826F52EC09F0A6C500F150
:1016D0000101003B0F0E0017F6EC1AF027C182F44F
:1016E0000401300E822752EC09F0A6C500F1010179
:1016F0000F0E01010017F6EC1AF027C182F4040165
:10170000300E822752EC09F004013A0E826F52EC3F
:1017100009F0A5C500F10101003B0F0E0017F6EC22
:101720001AF027C182F40401300E822752EC09F02E
:10173000A5C500F101010F0E0017F6EC1AF027C144
:1017400082F40401300E822752EC09F0120084C3A7
:10175000E8FF0F0BE83AE8CFABF585C3E8FF0F0BC6
:101760000501AB1387C3E8FF0F0BE83AE8CFAAF5F2
:1017700088C3E8FF0F0B0501AA138AC3E8FF0F0B0C
:10178000E83AE8CFA9F58BC3E8FF0F0B0501A913D1
:101790008DC3E8FF0F0BE8CFA8F58FC3E8FF0F0B51
:1017A000E83AE8CFA7F590C3E8FF0F0B0501A713B0
:1017B00092C3E8FF0F0BE83AE8CFA6F593C3E8FF22
:1017C0000F0B0501A61395C3E8FF0F0BE83AE8CF0E
:1017D000A5F596C3E8FF0F0B0501A5131FEC1CF040
:1017E00004014C0E826F52EC09F00401430E826F2B
:1017F00052EC09F0B9EF0AF0E4EC20F053EC1BF0E6
:101800002DC500F1F6EC1AF004014C0E826F52EC7B
:1018100009F00401300E826F52EC09F004012C0E25
:10182000826F52EC09F025C182F40401300E822748
:1018300052EC09F026C182F40401300E822752ECEA
:1018400009F027C182F40401300E822752EC09F01E
:1018500004012C0E826F52EC09F053EC1BF02EC5E4
:1018600000F1F6EC1AF025C182F40401300E822753
:1018700052EC09F026C182F40401300E822752ECAA
:1018800009F027C182F40401300E822752EC09F0DE
:10189000A2EF0DF004014C0E826F52EC09F004012E
:1018A000310E826F52EC09F004012C0E826F52EC63
:1018B00009F025C500F126C501F127C502F128C5AB
:1018C00003F10101100E046F000E056F000E066F8C
:1018D000000E076F8AEC1AF0F6EC1AF022C182F4BF
:1018E0000401300E822752EC09F023C182F4040176
:1018F000300E822752EC09F024C182F40401300E2C
:10190000822752EC09F025C182F40401300E8227AF
:1019100052EC09F026C182F40401300E822752EC09
:1019200009F027C182F40401300E822752EC09F03D
:10193000A2EF0DF04EEC1EF0E6EF14F004014C0E99
:10194000826F52EC09F00401330E826F52EC09F001
:1019500084EC1EF054EF0CF004014C0E826F52EC3C
:1019600009F00401340E826F52EC09F004012C0ED0
:10197000826F52EC09F094EC1BF084C31EF185C316
:101980001FF186C320F187C321F188C322F189C3E7
:1019900023F18AC324F18BC325F18CC326F18DC3B7
:1019A00027F101011D6BA1EC1BF018EC1BF0100ED0
:1019B000046F000E056F000E066F000E076F6BECD4
:1019C0001AF000C121F501C122F502C123F503C1BE
:1019D00024F597EC20F02EC5A5F52FC5A6F530C54A
:1019E000A7F531C5A8F532C5A9F533C5AAF534C5A3
:1019F000ABF5C4EC0AF004012C0E826F52EC09F036
:101A000035C500F136C501F137C502F138C503F11E
:101A10000101000E046F000E056F010E066F000E2F
:101A2000076F8AEC1AF0F6EC1AF01D671AEF0DF04A
:101A30001FEF0DF004012D0E826F52EC09F024C14E
:101A400082F40401300E822752EC09F025C182F4A1
:101A50000401300E822752EC09F004012E0E826F31
:101A600052EC09F026C182F40401300E822752ECB8
:101A700009F027C182F40401300E822752EC09F0EC
:101A800004012C0E826F52EC09F053EC1BF039C5A7
:101A900000F13AC501F110EC16F004012C0E826F32
:101AA00052EC09F053EC1BF03BC500F1F6EC1AF0D8
:101AB00025C182F40401300E822752EC09F026C1C0
:101AC00082F40401300E822752EC09F027C182F41F
:101AD0000401300E822752EC09F0A2EF0DF00E98AF
:101AE00084EC1EF0A2EF0DF004014C0E826F52EC5C
:101AF00009F00401350E826F52EC09F004012C0E3E
:101B0000826F52EC09F053EC1BF00784AFC500F173
:101B10000794F6EC1AF025C182F40401300E8227F6
:101B200052EC09F026C182F40401300E822752ECF7
:101B300009F027C182F40401300E822752EC09F02B
:101B4000A2EF0DF05CEC09F0E6EF14F004014C0E8E
:101B5000826F52EC09F00401500E826F52EC09F0D2
:101B600004012C0E826F52EC09F085C31EF186C36E
:101B70001FF187C320F188C321F189C322F18AC3F1
:101B800023F18BC324F18CC325F18DC326F18EC3C1
:101B900027F10101A1EC1BF018EC1BF003018451AB
:101BA000530A0DE0030184514D0A38E00401780E18
:101BB000826F52EC09F05CEC09F0E6EF14F00401DE
:101BC000530E826F52EC09F0250E0C6E00C10BF023
:101BD0009FEC06F0260E0C6E01C10BF09FEC06F098
:101BE000270E0C6E02C10BF09FEC06F0280E0C6E57
:101BF00003C10BF09FEC06F000C14DF501C14EF59D
:101C000002C14FF503C150F500C151F501C152F5B4
:101C100002C153F503C154F583EF0EF004014D0EDC
:101C2000826F52EC09F0290E0C6E00C10BF09FEC94
:101C300006F000C155F500C156F583EF0EF0040122
:101C40004C0E826F52EC09F00401540E826F52EC7C
:101C500009F004012C0E826F52EC09F084C31EF1CE
:101C600085C31FF186C320F187C321F188C322F108
:101C700089C323F18AC324F18BC325F18DC326F1D7
:101C80008EC327F10101A1EC1BF018EC1BF0010140
:101C9000000E046F000E056F010E066F000E076F39
:101CA0006BEC1AF0210E0C6E00C10BF09FEC06F0ED
:101CB000220E0C6E01C10BF09FEC06F0230E0C6E91
:101CC00002C10BF09FEC06F0240E0C6E03C10BF06A
:101CD0009FEC06F000C157F501C158F502C159F556
:101CE00003C15AF583EF0EF004014C0E826F52ECE3
:101CF00009F00401490E826F52EC09F004012C0E28
:101D0000826F52EC09F0250EB5EC06F0E8CF00F139
:101D1000260EB5EC06F0E8CF01F1270EB5EC06F083
:101D2000E8CF02F1280EB5EC06F0E8CF03F1F6ECAF
:101D30001AF022EC19F00401730E826F52EC09F0D4
:101D400004012C0E826F52EC09F053EC1BF0290EAB
:101D5000B5EC06F0E8CF00F1F6EC1AF022EC19F041
:101D60000401730E826F52EC09F004012C0E826F95
:101D700052EC09F051C500F152C501F153C502F111
:101D800054C503F1F6EC1AF022EC19F00401730EBD
:101D9000826F52EC09F004012C0E826F52EC09F0B4
:101DA00053EC1BF056C500F1F6EC1AF022EC19F0DA
:101DB00004016D0E826F52EC09F004012C0E826F4B
:101DC00052EC09F057C500F158C501F159C502F1AF
:101DD0005AC503F101EC15F004012C0E826F52EC90
:101DE00009F05CEC09F0E6EF14F083C31EF184C344
:101DF0001FF185C320F186C321F187C322F188C377
:101E000023F189C324F18AC325F18BC326F18CC346
:101E100027F10101A1EC1BF018EC1BF0160E0C6E63
:101E200000C10BF09FEC06F0170E0C6E01C10BF019
:101E30009FEC06F0180E0C6E02C10BF09FEC06F042
:101E4000190E0C6E03C10BF09FEC06F000C15DF1A2
:101E500001C15EF102C15FF103C160F100C161F136
:101E600001C162F102C163F103C164F1D7EF0FF068
:101E700083C31EF184C31FF185C320F186C321F102
:101E800087C322F188C323F189C324F18AC325F1D2
:101E90008BC326F18CC327F10101A1EC1BF018ECD8
:101EA0001BF000C15DF101C15EF102C15FF103C130
:101EB00060F100C161F101C162F102C163F103C1CE
:101EC00064F1D7EF0FF083C31EF184C31FF185C304
:101ED00020F186C321F187C322F188C323F189C38E
:101EE00024F18AC325F18CC326F18DC327F10101AA
:101EF000A1EC1BF018EC1BF00101000E046F000EAA
:101F0000056F010E066F000E076F6BEC1AF01A0ECC
:101F10000C6E00C10BF09FEC06F01B0E0C6E01C1A5
:101F20000BF09FEC06F01C0E0C6E02C10BF09FEC48
:101F300006F01D0E0C6E03C10BF09FEC06F000C105
:101F400065F101C166F102C167F103C168F1D7EF24
:101F50000FF083C31EF184C31FF185C320F186C334
:101F600021F187C322F188C323F189C324F18AC3F5
:101F700025F18CC326F18DC327F10101A1EC1BF0E3
:101F800018EC1BF00101000E046F000E056F010E2E
:101F9000066F000E076F6BEC1AF000C165F101C10E
:101FA00066F102C167F103C168F1D7EF0FF0160EB9
:101FB000B5EC06F0E8CF00F1170EB5EC06F0E8CF6F
:101FC00001F1180EB5EC06F0E8CF02F1190EB5ECF0
:101FD00006F0E8CF03F1F6EC1AF022EC19F0040158
:101FE000730E826F52EC09F004012C0E826F52ECDA
:101FF00009F05DC100F15EC101F15FC102F160C194
:1020000003F1F6EC1AF022EC19F00401730E826F62
:1020100052EC09F004012C0E826F52EC09F01A0EFA
:10202000B5EC06F0E8CF00F11B0EB5EC06F0E8CFFA
:1020300001F11C0EB5EC06F0E8CF02F11D0EB5EC77
:1020400006F0E8CF03F101EC15F004012C0E826FCD
:1020500052EC09F065C100F166C101F167C102F1FE
:1020600068C103F101EC15F05CEC09F0E6EF14F047
:102070000401690E826F52EC09F004012C0E826F8C
:1020800052EC09F00101040E006F000E016F000E0A
:10209000026F000E036FF6EC1AF020C182F4040107
:1020A000300E822752EC09F021C182F40401300E77
:1020B000822752EC09F022C182F40401300E8227FB
:1020C00052EC09F023C182F40401300E822752EC55
:1020D00009F024C182F40401300E822752EC09F089
:1020E00025C182F40401300E822752EC09F026C18A
:1020F00082F40401300E822752EC09F027C182F4E9
:102100000401300E822752EC09F004012C0E826F7C
:1021100052EC09F00101060E006F000E016F000E77
:10212000026F000E036FF6EC1AF020C182F4040176
:10213000300E822752EC09F021C182F40401300EE6
:10214000822752EC09F022C182F40401300E82276A
:1021500052EC09F023C182F40401300E822752ECC4
:1021600009F024C182F40401300E822752EC09F0F8
:1021700025C182F40401300E822752EC09F026C1F9
:1021800082F40401300E822752EC09F027C182F458
:102190000401300E822752EC09F004012C0E826FEC
:1021A00052EC09F00101140E006F000E016F000ED9
:1021B000026F000E036FF6EC1AF020C182F40401E6
:1021C000300E822752EC09F021C182F40401300E56
:1021D000822752EC09F022C182F40401300E8227DA
:1021E00052EC09F023C182F40401300E822752EC34
:1021F00009F024C182F40401300E822752EC09F068
:1022000025C182F40401300E822752EC09F026C168
:1022100082F40401300E822752EC09F027C182F4C7
:102220000401300E822752EC09F004012C0E826F5B
:1022300052EC09F0200EF86EF76AF66A0401090004
:10224000F5CF82F452EC09F00900F5CF82F452EC9C
:1022500009F00900F5CF82F452EC09F00900F5CF3E
:1022600082F452EC09F00900F5CF82F452EC09F047
:102270000900F5CF82F452EC09F00900F5CF82F4A1
:1022800052EC09F00900F5CF82F452EC09F05CEC55
:1022900009F0E6EF14F08351630AD8A4E6EF14F0D6
:1022A0008451610AD8A4E6EF14F085516C0AD8A4D1
:1022B000E6EF14F08651410A42E08651440A1BE0E1
:1022C0008651420AD8B4B2EF11F08651350AD8B41B
:1022D00070EF16F08651360AD8B4C5EF16F0865165
:1022E000370AD8B42EEF17F08651380AD8B48CEFDD
:1022F00017F0E6EF14F00798079A04017A0E826F40
:1023000052EC09F00401780E826F52EC09F00401DE
:10231000640E826F52EC09F081A896EF11F004016F
:10232000550E826F52EC09F09BEF11F004014C0E38
:10233000826F52EC09F05CEC09F0E6EF14F00788CC
:10234000079A04017A0E826F52EC09F00401410EE3
:10235000826F52EC09F00401610E826F52EC09F0B9
:102360008CEF11F00798078A04017A0E826F52EC05
:1023700009F00401420E826F52EC09F00401610E73
:10238000826F52EC09F08CEF11F00101620E046FC4
:10239000010E056F000E066F000E076F59C100F1A8
:1023A0005AC101F15BC102F15CC103F15CEC1AF0AE
:1023B00003BF22EF12F00E0EB5EC06F0E8CF0CF1E1
:1023C0000F0EB5EC06F0E8CF0DF1100EB5EC06F0EF
:1023D000E8CF0EF1110EB5EC06F0E8CF0FF1A5EC49
:1023E00019F059C104F15AC105F15BC106F15CC194
:1023F00007F15CEC1AF0078269EC19F0A5EC19F012
:10240000079269EC19F059C100F15AC101F15BC1A1
:1024100002F15CC103F1079269EC19F0CC0E046F74
:10242000E00E056F870E066F050E076F5CEC1AF065
:1024300000C10CF101C10DF102C10EF103C10FF198
:102440005AEF12F00101800E006F1A0E016F060E96
:10245000026F000E036F42C104F143C105F144C194
:1024600006F145C107F15CEC1AF003AF3BEF12F047
:1024700053EC1BF012000E0EB5EC06F0E8CF0CF199
:102480000F0EB5EC06F0E8CF0DF1100EB5EC06F02E
:10249000E8CF0EF1110EB5EC06F0E8CF0FF142C116
:1024A00000F143C101F144C102F145C103F10782CA
:1024B00069EC19F00CC100F10DC101F10EC102F17E
:1024C0000FC103F112000401730E826F52EC09F088
:1024D00004012C0E826F52EC09F0078455C159F1AA
:1024E00056C15AF157C15BF158C15CF13EC142F18E
:1024F0003FC143F140C144F141C145F14AC14CF1F2
:102500004BC14DF1079489EC12F05CEC09F0E6EF59
:1025100014F059C100F15AC101F15BC102F15CC173
:1025200003F10101F6EC1AF022EC19F00401630E3C
:10253000826F52EC09F004012C0E826F52EC09F00C
:1025400042C100F143C101F144C102F145C103F1AF
:102550000101F6EC1AF022EC19F00401660E826F0C
:1025600052EC09F004012C0E826F52EC09F053EC8E
:102570001BF04CC100F14DC101F10101F6EC1AF064
:1025800022EC19F00401740E826F52EC09F0120073
:102590000F820401530E826F52EC09F004012C0EDD
:1025A000826F52EC09F083C31EF184C31FF185C30F
:1025B00020F186C321F187C322F188C323F189C3A7
:1025C00024F18AC325F18BC326F18CC327F10101C5
:1025D000A1EC1BF018EC1BF000C159F101C15AF13C
:1025E00002C15BF103C15CF18EC31EF18FC31FF109
:1025F00090C320F191C321F192C322F193C323F13F
:1026000094C324F195C325F196C326F197C327F10E
:102610000101A1EC1BF018EC1BF000C142F101C15B
:1026200043F102C144F103C145F194EC1BF099C39D
:1026300023F19AC324F19BC325F19CC326F19DC3CA
:1026400027F10101A1EC1BF018EC1BF000C14CF1CB
:1026500001C14DF189EC12F004012C0E826F52EC95
:1026600009F03AEF13F08251520A03E10E823AEF79
:1026700013F00E9207840FB252EF13F055C159F1C7
:1026800056C15AF157C15BF158C15CF13EC142F1EC
:102690003FC143F140C144F141C145F14AC14CF150
:1026A0004BC14DF107940EA074EF13F00101656763
:1026B00061EF13F0666761EF13F0676761EF13F086
:1026C000686765EF13F074EF13F0C5EC11F065C1A6
:1026D00004F166C105F167C106F168C107F15CEC60
:1026E0001AF003BFAEEF14F0C5EC11F00101000EBB
:1026F000046F000E056F010E066F000E076F8AEC67
:102700001AF00401720E826F52EC09F004012C0ED3
:10271000826F52EC09F0F6EC1AF01D6795EF13F09A
:102720000401200E826F98EF13F004012D0E826FCA
:1027300052EC09F024C182F40401300E822752ECDD
:1027400009F025C182F40401300E822752EC09F011
:1027500004012E0E826F52EC09F026C182F40401AE
:10276000300E822752EC09F027C182F40401300EAA
:10277000822752EC09F004016D0E826F52EC09F0D1
:1027800004012C0E826F52EC09F042C100F143C1EA
:1027900001F144C102F145C103F10101F6EC1AF067
:1027A00022EC19F00401480E826F52EC09F004018A
:1027B0007A0E826F52EC09F004012C0E826F52ECFB
:1027C00009F059C100F15AC101F15BC102F15CC1CC
:1027D00003F10101F6EC1AF022EC19F00401630E8A
:1027E000826F52EC09F004012C0E826F52EC09F05A
:1027F00059C100F15AC101F15BC102F15CC103F1A1
:1028000001010A0E046F000E056F000E066F000E28
:10281000076F6BEC1AF0000E046F120E056F000EBE
:10282000066F000E076F8AEC1AF0F6EC1AF01EC164
:1028300082F40401300E822752EC09F01FC182F4A9
:102840000401300E822752EC09F020C182F4040109
:10285000300E822752EC09F021C182F40401300EBF
:10286000822752EC09F022C182F40401300E822743
:1028700052EC09F023C182F40401300E822752EC9D
:1028800009F024C182F40401300E822752EC09F0D1
:1028900004012E0E826F52EC09F025C182F404016E
:1028A000300E822752EC09F026C182F40401300E6A
:1028B000822752EC09F027C182F40401300E8227EE
:1028C00052EC09F00401730E826F52EC09F004011E
:1028D0002C0E826F52EC09F053EC1BF04CC100F14E
:1028E0004DC101F110EC16F00EB27AEF14F00EA00B
:1028F000ACEF14F004012C0E826F52EC09F0200EA4
:10290000F86EF76AF66A04010900F5CF82F452EC1A
:1029100009F00900F5CF82F452EC09F00900F5CF77
:1029200082F452EC09F00900F5CF82F452EC09F080
:102930000900F5CF82F452EC09F00900F5CF82F4DA
:1029400052EC09F00900F5CF82F452EC09F00900CD
:10295000F5CF82F452EC09F05CEC09F00E90E6EF52
:1029600014F00401630E826F52EC09F004012C0E86
:10297000826F52EC09F0ECEC14F004012C0E826F23
:1029800052EC09F05FEC15F004012C0E826F52EC52
:1029900009F0DBEC15F004012C0E826F52EC09F00B
:1029A0000101F80E006FCD0E016F660E026F030E6F
:1029B000036F01EC15F004012C0E826F52EC09F04C
:1029C000F1EC15F05CEC09F0E6EF14F00301A26BFA
:1029D00007900F92F5EF17F0D8900E0EB5EC06F0B9
:1029E000E8CF00F10F0EB5EC06F0E8CF01F1100EC4
:1029F000B5EC06F0E8CF02F1110EB5EC06F0E8CF29
:102A000003F10101000E046F000E056F010E066F49
:102A1000000E076F8AEC1AF0F6EC1AF01EC182F471
:102A20000401300E822752EC09F01FC182F4040128
:102A3000300E822752EC09F020C182F40401300EDE
:102A4000822752EC09F021C182F40401300E822762
:102A500052EC09F022C182F40401300E822752ECBC
:102A600009F023C182F40401300E822752EC09F0F0
:102A700024C182F40401300E822752EC09F025C1F2
:102A800082F40401300E822752EC09F004012E0E6C
:102A9000826F52EC09F026C182F40401300E8227C5
:102AA00052EC09F027C182F40401300E822752EC67
:102AB00009F004016D0E826F52EC09F01200120E43
:102AC000B5EC06F0E8CF00F1130EB5EC06F0E8CF58
:102AD00001F1140EB5EC06F0E8CF02F1150EB5ECDD
:102AE00006F0E8CF03F101010A0E046F000E056F36
:102AF000000E066F000E076F6BEC1AF0000E046FED
:102B0000120E056F000E066F000E076F8AEC1AF0AA
:102B1000F6EC1AF01EC182F40401300E822752EC4A
:102B200009F01FC182F40401300E822752EC09F033
:102B300020C182F40401300E822752EC09F021C139
:102B400082F40401300E822752EC09F022C182F493
:102B50000401300E822752EC09F023C182F40401F3
:102B6000300E822752EC09F024C182F40401300EA9
:102B7000822752EC09F004012E0E826F52EC09F00C
:102B800025C182F40401300E822752EC09F026C1DF
:102B900082F40401300E822752EC09F027C182F43E
:102BA0000401300E822752EC09F00401730E826F8B
:102BB00052EC09F012000A0EB5EC06F0E8CF00F175
:102BC0000B0EB5EC06F0E8CF01F10C0EB5EC06F0FB
:102BD000E8CF02F10D0EB5EC06F0E8CF03F110EFEF
:102BE00016F0060EB5EC06F0E8CF00F1070EB5ECD6
:102BF00006F0E8CF01F1080EB5EC06F0E8CF02F1DF
:102C0000090EB5EC06F0E8CF03F110EF16F0010164
:102C100053EC1BF007844AC100F14BC101F107944A
:102C20000101E80E046F800E056F000E066F000EA6
:102C3000076F6BEC1AF0000E046F040E056F000EA8
:102C4000066F000E076F8AEC1AF0880E046F130EE1
:102C5000056F000E066F000E076F5CEC1AF00A0E8F
:102C6000046F000E056F000E066F000E076F8AECF2
:102C70001AF0F6EC1AF001011D6744EF16F004019A
:102C8000200E826F47EF16F004012D0E826F52EC7A
:102C900009F024C182F40401300E822752EC09F0BD
:102CA00025C182F40401300E822752EC09F026C1BE
:102CB00082F40401300E822752EC09F004012E0E3A
:102CC000826F52EC09F027C182F40401300E822792
:102CD00052EC09F00401430E826F52EC09F012002D
:102CE00087C31EF188C31FF189C320F18AC321F174
:102CF0008BC322F18CC323F18DC324F18EC325F144
:102D000090C326F191C327F101011D6BA1EC1BF0CB
:102D100018EC1BF00101000E046F000E056F010E90
:102D2000066F000E076F6BEC1AF00E0E0C6E00C1F2
:102D30000BF09FEC06F00F0E0C6E01C10BF09FEC38
:102D400006F0100E0C6E02C10BF09FEC06F0110E97
:102D50000C6E03C10BF09FEC06F004017A0E826F3B
:102D600052EC09F004012C0E826F52EC09F00401C0
:102D7000350E826F52EC09F004012C0E826F52EC7A
:102D800009F0ECEC14F09BEF11F087C31EF188C33F
:102D90001FF189C320F18AC321F18BC322F18CC3B7
:102DA00023F18DC324F18EC325F190C326F191C385
:102DB00027F101011D6BA1EC1BF018EC1BF0880E34
:102DC000046F130E056F000E066F000E076F60ECA8
:102DD0001AF0000E046F040E056F000E066F000E51
:102DE000076F6BEC1AF00101E80E046F800E056F9F
:102DF000000E066F000E076F8AEC1AF00A0E0C6EBA
:102E000000C10BF09FEC06F00B0E0C6E01C10BF035
:102E10009FEC06F00C0E0C6E02C10BF09FEC06F05E
:102E20000D0E0C6E03C10BF09FEC06F004017A0E40
:102E3000826F52EC09F004012C0E826F52EC09F003
:102E40000401360E826F52EC09F004012C0E826FE1
:102E500052EC09F0DBEC15F09BEF11F087C31EF18B
:102E600088C31FF189C320F18AC321F18BC322F1EA
:102E70008CC323F18DC324F18FC325F190C326F1B8
:102E800091C327F10101A1EC1BF018EC1BF0000E1F
:102E9000046F120E056F000E066F000E076F6BECCD
:102EA0001AF001010A0E046F000E056F000E066F86
:102EB000000E076F8AEC1AF0120E0C6E00C10BF0B8
:102EC0009FEC06F0130E0C6E01C10BF09FEC06F0A8
:102ED000140E0C6E02C10BF09FEC06F0150E0C6E7A
:102EE00003C10BF09FEC06F004017A0E826F52ECE6
:102EF00009F004012C0E826F52EC09F00401370E28
:102F0000826F52EC09F004012C0E826F52EC09F032
:102F10005FEC15F09BEF11F087C31EF188C31FF122
:102F200089C320F18AC321F18BC322F18CC323F121
:102F30008DC324F18EC325F190C326F191C327F1EF
:102F400001011D6BA1EC1BF018EC1BF0880E046F47
:102F5000130E056F000E066F000E076F60EC1AF07F
:102F6000000E046F040E056F000E066F000E076F53
:102F70006BEC1AF00101E80E046F800E056F000E75
:102F8000066F000E076F8AEC1AF0060E0C6E00C179
:102F90000BF09FEC06F0070E0C6E01C10BF09FECDE
:102FA00006F0080E0C6E02C10BF09FEC06F0090E45
:102FB0000C6E03C10BF09FEC06F004017A0E826FD9
:102FC00052EC09F004012C0E826F52EC09F004015E
:102FD000380E826F52EC09F004012C0E826F52EC15
:102FE00009F0F1EC15F09BEF11F081A8B3EF18F0A8
:102FF00007A86CEF18F00101800E006F1A0E016F28
:10300000060E026F000E036F3EC104F13FC105F1D1
:1030100040C106F141C107F15CEC1AF003BFB3EF08
:1030200018F01CEC19F03EC100F13FC101F140C1A4
:1030300002F141C103F1078269EC19F00CC104F1FE
:103040000DC105F10EC106F10FC107F1F80E006FB9
:10305000CD0E016F660E026F030E036F5CEC1AF06B
:103060000E0E0C6E00C10BF09FEC06F00F0E0C6EF6
:1030700001C10BF09FEC06F0100E0C6E02C10BF0BC
:103080009FEC06F0110E0C6E03C10BF09FEC06F0E6
:103090000784010153EC1BF04AC100F14BC101F15F
:1030A00007940A0E0C6E00C10BF09FEC06F00B0E9D
:1030B0000C6E01C10BF09FEC06F00C0E0C6E02C101
:1030C0000BF09FEC06F00D0E0C6E03C10BF09FECA5
:1030D00006F00798B3EF18F007AAB3EF18F00784CB
:1030E000010153EC1BF04AC100F14BC101F10794FF
:1030F000060E0C6E00C10BF09FEC06F0070E0C6E76
:1031000001C10BF09FEC06F0080E0C6E02C10BF033
:103110009FEC06F0090E0C6E03C10BF09FEC06F05D
:10312000078455C100F156C101F157C102F158C1E0
:1031300003F10794120E0C6E00C10BF09FEC06F029
:10314000130E0C6E01C10BF09FEC06F0140E0C6E0A
:1031500002C10BF09FEC06F0150E0C6E03C10BF0D4
:103160009FEC06F0079A0401805181197F0B0BE058
:103170009EA809D014EE00F081517F0BE126E750A4
:10318000812B0F01AD6E05012951010A13E081AABF
:10319000DAEF18F005012951000A0AE00EB8DAEF5B
:1031A00018F005012A67DAEF18F00EB8DAEF18F018
:1031B00023EF21F081B8EEEF18F070EC1CF0050160
:1031C0002951020A02E0EEEF18F0562FEEEF18F048
:1031D00055C556F50501060E2A6F2B6BC5EF08F095
:1031E0000CC100F10DC101F10EC102F10FC103F1DB
:1031F000000E046F000E056F010E066F000E076FC4
:103200008AEC1AF01DA11BEF19F01451D8B41BEF72
:1032100019F00CC100F10DC101F10EC102F10FC195
:1032200003F1000E046F000E056F0A0E066F000E0C
:10323000076F8AEC1AF0120001010C6B0D6B0E6B1C
:103240000F6B12001EC182F40401300E822752EC73
:1032500009F01FC182F40401300E822752EC09F0FC
:1032600020C182F40401300E822752EC09F021C102
:1032700082F40401300E822752EC09F022C182F45C
:103280000401300E822752EC09F023C182F40401BC
:10329000300E822752EC09F024C182F40401300E72
:1032A000822752EC09F025C182F40401300E8227F6
:1032B00052EC09F026C182F40401300E822752EC50
:1032C00009F027C182F40401300E822752EC09F084
:1032D00012000101005305E1015303E1025301E132
:1032E000002B2CEC1AF053EC1BF02C51006F2D51DD
:1032F000016F420E046F4B0E056F000E066F000E3D
:10330000076F6BEC1AF000C104F101C105F102C1B5
:1033100006F103C107F10CC100F10DC101F10EC1AD
:1033200002F10FC103F107B29AEF19F060EC1AF045
:103330009CEF19F05CEC1AF000C10CF101C10DF129
:1033400002C10EF103C10FF1120053EC1BF04CC18E
:1033500000F14DC101F1060EB5EC06F0E8CF04F125
:10336000070EB5EC06F0E8CF05F1080EB5EC06F057
:10337000E8CF06F1090EB5EC06F0E8CF07F15CECFA
:103380001AF000C118F101C119F102C11AF103C10B
:103390001BF1290E046F000E056F000E066F000E64
:1033A000076F6BEC1AF0EE0E046F430E056F000E04
:1033B000066F000E076F60EC1AF018C104F119C116
:1033C00005F11AC106F11BC107F16BEC1AF000C13F
:1033D00010F101C111F102C112F103C113F1120E7A
:1033E000B5EC06F0E8CF04F1130EB5EC06F0E8CF2B
:1033F00005F1140EB5EC06F0E8CF06F1150EB5ECAC
:1034000006F0E8CF07F10D0E006F000E016F000E01
:10341000026F000E036F6BEC1AF0180E046F000EB3
:10342000056F000E066F000E076F8AEC1AF010C1D0
:1034300004F111C105F112C106F113C107F160ECED
:103440001AF06A0E046F2A0E056F000E066F000E4A
:10345000076F5CEC1AF01200BF0EFA6E200E2D6F93
:103460002C6BD8900037013702370337D8B03DEFC7
:103470001AF02D2F32EF1AF02C072D070353D8B472
:1034800012000331070B8009326F03390F0B010F54
:103490002C6F80EC5FF0336F2C0580EC5FF0335DB8
:1034A000335F2C6B3233D8B02C272C3332A952EF38
:1034B0001AF033512C27120078EC1BF0D8B0120010
:1034C00003510719286F3BEC1BF0D89007510319E3
:1034D00028AF800F1200286B5FEC1BF0D8A075ECB2
:1034E0001BF0D8B012004AEC1BF053EC1BF01F0E7F
:1034F000296F8BEC1BF00B35D8B03BEC1BF0D8A040
:103500000335D8B01200292F79EF1AF028B162ECF8
:103510001BF01200286B0451051106110711000859
:10352000D8A05FEC1BF0D8A075EC1BF0D8B012004F
:10353000086B096B0A6B0B6B8BEC1BF01F0E296F72
:103540008BEC1BF007510B5DD8A4B3EF1AF00651BA
:103550000A5DD8A4B3EF1AF00551095DD8A4B3EF02
:103560001AF00451085DD8A0C6EF1AF00451085FA4
:103570000551D8A0053D095F0651D8A0063D0A5F58
:103580000751D8A0073D0B5FD8900081292FA0EFED
:103590001AF028B162EC1BF0286B5FEC1BF0D8909E
:1035A0008FEC1BF007510B5DD8A4E3EF1AF0065126
:1035B0000A5DD8A4E3EF1AF00551095DD8A4E3EF42
:1035C0001AF00451085DD8A0F2EF1AF0003FF2EFB4
:1035D0001AF0013FF2EF1AF0023FF2EF1AF0032B5C
:1035E000D8B4120028B162EC1BF012000101286B64
:1035F0005FEC1BF0D8B0120094EC1BF0200E296F8A
:10360000003701370237033711EE27F00A0E2A6F11
:10361000E7360A0EE75CD8B0E76EE5522A2F08EFCE
:103620001BF0292F00EF1BF028B11D81D89012004C
:1036300001010A0E286F200E296F11EE1DF028518E
:103640002A6F0A0ED890E652D8B0E726E7322A2F22
:1036500023EF1BF00333023301330033292F1DEF17
:103660001BF0E750FF0FD8A00335D8B012001DB1F2
:1036700062EC1BF01200045100270551D8B0053D43
:1036800001270651D8B0063D02270751D8B0073DA3
:10369000032712000051086F0151096F02510A6F90
:1036A00003510B6F12000101006B016B026B036B86
:1036B00012000101046B056B066B076B12000335EA
:1036C000D8A012000351800B001F011F021F031F0F
:1036D000003F72EF1BF0013F72EF1BF0023F72EFF1
:1036E0001BF0032B282B032512000735D8A012004E
:1036F0000751800B041F051F061F071F043F88EF9B
:103700001BF0053F88EF1BF0063F88EF1BF0072BEF
:10371000282B0725120000370137023703370837F7
:1037200009370A370B37120001011D6B1E6B1F6B27
:10373000206B216B226B236B246B256B266B276B15
:1037400012001E510F0B1E6F1F510F0B1F6F2051C8
:103750000F0B206F21510F0B216F22510F0B226F86
:1037600023510F0B236F24510F0B246F25510F0B87
:10377000256F26510F0B266F27510F0B276F120055
:103780008984000EC76E220EC66E9E96C69E000EDF
:10379000C96EFF0E9EB602D0E82EFCD79E96C69E3E
:1037A000000EC96EFF0E9EB602D0E82EFCD7C9CF20
:1037B000A5F59E96C69E000EC96EFF0E9EB602D05F
:1037C000E82EFCD7C9CFA6F59E96C69E000EC96E00
:1037D000FF0E9EB602D0E82EFCD7C9CFA7F59E9665
:1037E000C69E000EC96EFF0E9EB602D0E82EFCD714
:1037F000C9CFA8F59E96C69E000EC96EFF0E9EB656
:1038000002D0E82EFCD7C9CFA9F59E96C69E000E21
:10381000C96EFF0E9EB602D0E82EFCD7C9CFAAF51E
:103820009E96C69E000EC96EFF0E9EB602D0E82E72
:10383000FCD7C9CFABF5899400EC1EF01200898447
:10384000000EC76E220EC66E9E96C69E800EC96E74
:10385000FF0E9EB602D0E82EFCD79E96C69EA5C54A
:10386000C9FFFF0E9EB602D0E82EFCD79E96C69EDC
:10387000A6C5C9FFFF0E9EB602D0E82EFCD79E96C5
:10388000C69EA7C5C9FFFF0E9EB602D0E82EFCD784
:103890009E96C69EA8C5C9FFFF0E9EB602D0E82E12
:1038A000FCD79E96C69EA9C5C9FFFF0E9EB602D044
:1038B000E82EFCD79E96C69EAAC5C9FFFF0E9EB6EF
:1038C00002D0E82EFCD79E96C69EABC5C9FFFF0E60
:1038D0009EB602D0E82EFCD7899400EC1EF01200B0
:1038E0008984000EC76E220EC66E9E96C69E070E77
:1038F000C96EFF0E9EB602D0E82EFCD79E96C69EDD
:10390000000EC96EFF0E9EB602D0E82EFCD7C9CFBE
:10391000A5F59E96C69E000EC96EFF0E9EB602D0FD
:10392000E82EFCD7C9CFA6F59E96C69E000EC96E9E
:10393000FF0E9EB602D0E82EFCD7C9CFA7F59E9603
:10394000C69E000EC96EFF0E9EB602D0E82EFCD7B2
:10395000C9CFA8F5899400EC1EF08984000EC76ECB
:10396000220EC66E9E96C69E0F0EC96EFF0E9EB6A6
:1039700002D0E82EFCD79E96C69E000EC96EFF0EA2
:103980009EB602D0E82EFCD7C9CFADF5899400ECE5
:103990001EF012008984000EC76E220EC66E9E961F
:1039A000C69E870EC96EFF0E9EB602D0E82EFCD7CB
:1039B0009E96C69EA5C5C9FFFF0E9EB602D0E82EF4
:1039C000FCD79E96C69EA6C5C9FFFF0E9EB602D026
:1039D000E82EFCD79E96C69EA7C5C9FFFF0E9EB6D1
:1039E00002D0E82EFCD79E96C69EA8C5C9FFFF0E42
:1039F0009EB602D0E82EFCD7899400EC1EF0898494
:103A00009E96C69E8F0EC96EFF0E9EB602D0E82E01
:103A1000FCD79E96C69EADC5C9FFFF0E9EB602D0CE
:103A2000E82EFCD7899400EC1EF012008984000E69
:103A3000C76E220EC66E9E96C69E870EC96EFF0E7C
:103A40009EB602D0E82EFCD79E96C69E000EC96E8A
:103A5000FF0E9EB602D0E82EFCD79E96C69E800E24
:103A6000C96EFF0E9EB602D0E82EFCD79E96C69E6B
:103A7000800EC96EFF0E9EB602D0E82EFCD79E9631
:103A8000C69E800EC96EFF0E9EB602D0E82EFCD7F1
:103A9000899400EC1EF089849E96C69E8F0EC96E96
:103AA000FF0E9EB602D0E82EFCD79E96C69E010E53
:103AB000C96EFF0E9EB602D0E82EFCD7899400ECAA
:103AC0001EF012008984000EC76E220EC66E9E96EE
:103AD000C69E870EC96EFF0E9EB602D0E82EFCD79A
:103AE0009E96C69E000EC96EFF0E9EB602D0E82EB0
:103AF000FCD79E96C69E000EC96EFF0E9EB602D0E3
:103B0000E82EFCD79E96C69E800EC96EFF0E9EB60E
:103B100002D0E82EFCD79E96C69E800EC96EFF0E80
:103B20009EB602D0E82EFCD7899400EC1EF0898462
:103B30009E96C69E8F0EC96EFF0E9EB602D0E82ED0
:103B4000FCD79E96C69E010EC96EFF0E9EB602D091
:103B5000E82EFCD7899400EC1EF012008984000E38
:103B6000C76E220EC66E9E96C69E8F0EC96EFF0E43
:103B70009EB602D0E82EFCD700EC1EF09E96C69EA4
:103B8000010EC96EFF0E9EB602D0E82EFCD78994B6
:103B900000EC1EF089849E96C69E910EC96EFF0EA3
:103BA0009EB602D0E82EFCD700EC1EF09E96C69E74
:103BB000A50EC96EFF0E9EB602D0E82EFCD78994E2
:103BC00000EC1EF012008984000EC76E220EC66E35
:103BD0009E96C69E910EC96EFF0E9EB602D0E82E2E
:103BE000FCD700EC1EF09E96C69E000EC96EFF0E1E
:103BF0009EB602D0E82EFCD7899400EC1EF012008D
:103C0000050EE82EFED71200200EC66E0501256BAC
:103C1000266B276B286B899A400EC76E200EC66EE6
:103C20009E96C69E030EC96EFF0E9EB602D0E82E6B
:103C3000FCD79E96C69E27C5C9FFFF0E9EB602D032
:103C4000E82EFCD79E96C69E26C5C9FFFF0E9EB6DF
:103C500002D0E82EFCD79E96C69E25C5C9FFFF0E52
:103C60009EB602D0E82EFCD79E96C69EC952FF0E85
:103C70009EB602D0E82EFCD7898AC950FF0A02E11D
:103C80004BEF1EF0100E2527E86A2623E86A27234B
:103C900027A90BEF1EF0220EC66E1200899A400E65
:103CA000C76E200EC66E9E96C69E060EC96EFF0E8D
:103CB0009EB602D0E82EFCD7898A899A9E96C69E27
:103CC000C70EC96EFF0E9EB602D0E82EFCD7898AB9
:103CD000899A9E96C69E050EC96EFF0E9EB602D0AC
:103CE000E82EFCD79E96C69EC952FF0E9EB602D005
:103CF000E82EFCD7C9B072EF1EF0898A0501256B4A
:103D0000266B276B286B12000501FE0E2D6F050137
:103D1000000E2D6FC0EC1BF0A5C52EF5A6C52FF526
:103D2000A7C530F5A8C531F5A9C532F5AAC533F543
:103D3000ABC534F5078455C159F156C15AF157C185
:103D40005BF158C15CF13EC142F13FC143F140C15A
:103D500044F141C145F14AC14CF14BC14DF10794C9
:103D6000C5EC11F000C135F501C136F502C137F5DA
:103D700003C138F505015767C5EF1EF05867C5EF59
:103D80001EF05967C5EF1EF05A67C9EF1EF0D7EF56
:103D90001EF057C504F158C505F159C506F15AC5BD
:103DA00007F101015CEC1AF003BF45EF1FF04CC1B5
:103DB00039F54DC13AF5AFC53BF5B0C53CF5050148
:103DC000100E2C6F899A400EC76E200EC66E9E96FE
:103DD000C69E060EC96EFF0E9EB602D0E82EFCD718
:103DE000898A899A9E96C69E020EC96EFF0E9EB65D
:103DF00002D0E82EFCD79E96C69E27C5C9FFFF0EAF
:103E00009EB602D0E82EFCD79E96C69E26C5C9FF58
:103E1000FF0E9EB602D0E82EFCD79E96C69E25C504
:103E2000C9FFFF0E9EB602D0E82EFCD725EE2DF07E
:103E30002C2F02D027EF1FF09E96C69EDECFC9FF23
:103E4000FF0E9EB602D0E82EFCD718EF1FF0898A2D
:103E5000899A9E96C69E050EC96EFF0E9EB602D02A
:103E6000E82EFCD79E96C69EC952FF0E9EB602D083
:103E7000E82EFCD7C9B032EF1FF0898A0501100E79
:103E80002527E86A2623E86A2723120019C502F5C8
:103E90001AC503F525EE5FF005012C6B16EE00F058
:103EA00005010251E1260351D8B00329E226E7CFEC
:103EB000E8FF2C0A06E12CC5DEFF05012C6B69EF3B
:103EC0001FF0E7CFE8FF2A0A0CE0E7CFDEFF05018D
:103ED0002C2B0501032B023F0307030E03174EEFA4
:103EE0001FF005012D6B2E6B2F6B306B316B326B1E
:103EF000336B346B356B366B376B386B396B3A6BB6
:103F00003B6B3C6B3D6B3E6B3F6B406B416B426B65
:103F1000436B446B456B466B476B486B496B4A6B15
:103F20004B6B4C6BDDCFE8FF05012C5105E0DDCF7D
:103F3000E8FF2C2F97EF1FF00501DDCF2CF52C515A
:103F400005E0DDCFE8FF2C2FA1EF1FF00501DDCF4D
:103F50002CF52C5105E0DDCFE8FF2C2FABEF1FF047
:103F600011EE27F0010194EC1BF00501DDCF2CF5DB
:103F70002C5105E0DDCFE5FF2C2FBAEF1FF001013A
:103F8000A1EC1BF018EC1BF000C12EF501C12FF5C0
:103F900002C130F50501DDCF2CF52C5105E0DDCF58
:103FA000E8FF2C2FCFEF1FF00501DDCF2CF52C51B2
:103FB00005E0DDCFE8FF2C2FD9EF1FF00501DDCFA5
:103FC0002CF52C5107E0DDCFE8FFE8A82D852C2F3C
:103FD000E3EF1FF011EE27F0010194EC1BF0050157
:103FE000DDCF2CF52C5114E0DDCFE5FFDDCFE5FF73
:103FF000DDCFE5FFDDCFE5FFDDCFE8FFDDCFE5FF7E
:10400000DDCFE5FFDDCFE5FFDDCFE5FFDDCFE5FF70
:104010000101A1EC1BF018EC1BF000C138F501C147
:1040200039F502C13AF503C13BF50501DDCF2CF5A9
:104030002C5107E0DDCFE8FFE8A82D832C2F1AEFE5
:1040400020F011EE27F0010194EC1BF00501DDCF0B
:104050002CF52C5105E0DDCFE5FF2C2F2BEF20F0C8
:10406000010122C123F121C122F120C121F11FC18F
:1040700020F1A1EC1BF018EC1BF000C134F501C1DC
:1040800035F502C136F503C137F50501DDCF2CF555
:104090002C5107E0DDCFE8FF2C2F4AEF20F0E8B0ED
:1040A0002D8711EE27F0010194EC1BF0DDCFE8FF26
:1040B000DDCFE8FFDDCFE8FFDDCFE8FFDDCFE8FFB4
:1040C000DDCFE5FFDDCFE5FFDDCFE5FFDDCFE5FFB0
:1040D000DDCFE5FFDDCFE5FFA1EC1BF018EC1BF019
:1040E00000C131F501C132F502C133F5078455C174
:1040F00059F156C15AF157C15BF158C15CF13EC14B
:1041000042F13FC143F140C144F141C145F14AC1CF
:104110004CF14BC14DF10794C5EC11F000C13CF5D9
:1041200001C13DF502C13EF503C13FF5120021C5B5
:1041300000F122C501F123C502F124C503F1899ADA
:10414000400EC76E200EC66E9E96C69E0B0EC96EA2
:10415000FF0E9EB602D0E82EFCD79E96C69E02C1E8
:10416000C9FFFF0E9EB602D0E82EFCD79E96C69ED3
:1041700001C1C9FFFF0E9EB602D0E82EFCD79E9665
:10418000C69E00C1C9FFFF0E9EB602D0E82EFCD726
:104190009E96C69EC952FF0E9EB602D0E82EFCD750
:1041A00025EE2DF00501100E2C6F9E96C69EC9526D
:1041B000FF0E9EB602D0E82EFCD7C9CFDEFF2C2F13
:1041C000D5EF20F0898A1200899A400EC76E200E22
:1041D000C66E9E96C69E900EC96EFF0E9EB602D00B
:1041E000E82EFCD79E96C69E000EC96EFF0E9EB6A8
:1041F00002D0E82EFCD79E96C69E000EC96EFF0E1A
:104200009EB602D0E82EFCD79E96C69E000EC96EC2
:10421000FF0E9EB602D0E82EFCD79E96C69EC952CF
:10422000FF0E9EB602D0E82EFCD7C9CF2DF59E9684
:10423000C69EC952FF0E9EB602D0E82EFCD7C9CF4B
:104240002EF5898A120070EC1CF0F29CF29E8B9481
:104250008A86899CC69AC2908A94898A9482948C10
:10426000720ED36ED3A4FED789968A909390FF0ED8
:10427000E8CF00F0E82EFED7002EFCD78150F29454
:10428000F29A9E909D909E929D92F298F292F29058
:08429000F286F28E0300FF002C
:10BF0000E844F926000C160C2B0C3F0C520C640C68
:10BF1000760C860C960CA50CB30CC10CCF0CDC0C6B
:06BF2000E80CF40C000C1B
:00000001FF
